:020000040000FA
:1000000000306500FF30660090019101920193017C
:100010009401950196019701980110081202031CA2
:100020001328851414288510900A031918200D2808
:1000300026201318910A3320141891034020151814
:10004000910111089A004D209200080086182B2873
:10005000960193013228161831280130960093003A
:1000600032289301080006193828970194013F2887
:1000700017183E280130970094003F28940108008B
:1000800086194528980195014C2818184B280130ED
:10009000980095004C2895010800803099001A08B6
:1000A00019020318572899008030190208001A080D
:0200B000080046
:02400E00F23F7F
:00000001FF
